:040000000200833245
:01000B0032C2
:0100130032BA
:01001B0032B2
:0100230032AA
:01002B0032A2
:01003300329A
:01003B003292
:01004300328A
:03004B000201515E
:01005300327A
:01005B003272
:01006300326A
:01006B003262
:01007300325A
:03007B000201D9A6
:1000DC00E4F521F522F523F524E4F525F526F5279D
:1000EC00752800752900752A01752B00E4F52CF58F
:1000FC002DF52EF52F753000E4F531F532F533750D
:10010C003506E4F539F53AF53BF53C753D00753EA1
:04011C000002007E5F
:05007E0012061E80FEC9
:1001200053BEFBE5BE30E6FB53C6B8E5C620E6FB92
:1001300043BE042275E40075DB3275DAC875E50448
:1001400075E60075E70075E200D2DED2B975E4020B
:1001500022C020C0E0C0F0C082C083C002C003C083
:1001600004C005C006C007C000C001C0D075D000E3
:1001700074012521F521E43522F522E43523F52308
:10018000E43524F524120327120218D0D0D001D070
:1001900000D007D006D005D004D003D002D083D041
:1001A00082D0F0D0E0D0203275860075C22275C5AD
:1001B0002D228582C1E58630E1FB5386FD85C18213
:1001C0002243F32843FD505380EBC2EB439A104384
:1001D0008D0243FE015390FE22C0E0E58A758A003D
:1001E000D0E032AA827B001AEA600A8B041CECFB86
:1001F00060F50080F82285820985830A85F00B75F9
:100200003405850931850A32850B33850836753505
:100210000075370043900122E535FA24F950012298
:10022000EA2A2A9002277302023C02026502028730
:100230000202AE0202EA0203010203017582001209
:1002400001B2AA82BAFA04753501221534E5346088
:10025000012275300185213985223A85233B852489
:100260003C753504227582001201B2AA82BAFB04E1
:100270007535022275300285213985223A85233B66
:1002800085243C753504227582001201B2858237BF
:100290007538005390FEE5376004753503228521DB
:1002A0003985223A85233B85243C75350422AA38BA
:1002B0000538EA2531FAE43532FBAC33758200C0EB
:1002C00002C003C0041201B2AD82D004D003D00238
:1002D0008A828B838CF0ED1206DAE537B53802801E
:1002E00005E536B5381B75350622C3E5219539E598
:1002F00022953AE523953BE524953C400475350568
:10030000222285820985830A85F00B74FC2508402A
:1003100003750804850925850A26850B2785082885
:10032000752B00752A0222E52AFA24F8500122EAE8
:100330002A2A9003367302034E02036E02036F02F1
:10034000037E02038B0203950203A20203B4E52B92
:100350006018C3E521952CE522952DE523952EE522
:1003600024952F500122752A0122752A0122227418
:10037000025590FABA0202800122752A0322758280
:10038000FA1201B285822B752A04227582FB1201B2
:10039000B2752A05228528821201B2752900752AB4
:1003A000062274025590FABA02028004752A0722C6
:1003B000752A0322AA290529EA2525FAE43526FB10
:1003C000AC278A828B838CF01206F3F5821201B27D
:1003D000E528B5291874C82521F52CE43522F52D1A
:1003E000E43523F52EE43524F52F752A0022AA8260
:1003F000AB83ACF01206F3FD7E0053057FBD010612
:10040000BE00030204ACBD0205BE00028013BD03A2
:1004100005BE0002805ABD0505BE0002802102040F
:10042000AC74012AFDE43BFE8C078D828E838FF035
:100430001206F360055380BF8072438040806D7563
:10044000E104758210C002C003C0041201E3D004AD
:10045000D003D00274012AFDE43BFE8C078D828E0E
:10046000838FF01206F3FD90DF06F075E103803C08
:1004700074012AFDE43BFE8C078D828E838FF0127F
:1004800006F3FE7D0074022AFFE43BF88C018F82A4
:10049000888389F01206F3FF78004205E842068D52
:1004A000428E43854282854383E0F53E8A828B8378
:1004B0008CF01206F3FD30E71C8A828B838CF0747B
:1004C000011206DAAD3FAE40AF418D828E838FF0D0
:1004D00074010206DA8A828B838CF0E41206DAAAAF
:1004E0003FAB40AC418A828B838CF074010206DA08
:1004F00090DF0074D3F090DF017491F090DF02740C
:10050000FFF090DF037404F090DF047422F090DFBA
:1005100005E4F090DF06F090DF077406F090DF0846
:10052000E4F090DF097421F090DF0A7465F090DF49
:100530000B746AF090DF0C74F5F090DF0D7483F0AB
:1005400090DF0E7410F090DF0F7422F090DF1074C3
:10055000F8F090DF117415F090DF127407F090DF5F
:10056000137430F090DF147418F090DF157417F0E6
:1005700090DF16746CF090DF177403F090DF18743E
:1005800040F090DF197491F090DF1A7456F090DF0C
:100590001B7410F090DF1C74E9F090DF1D742AF0DA
:1005A00090DF1EE4F090DF1F741FF090DF2374884B
:1005B000F090DF247431F090DF257409F090DF278C
:1005C000E4F090DF28F090DF29F090DF2AF090DF50
:1005D0002BE4F090DF2CF090DF2DF090DF2E74C232
:1005E000F090DF2FE4F090DF30F090DF31F090DF1B
:1005F000367401F090DF377403F090DF38E4F09048
:10060000DF3974FFF090DF3A7480F090DF3B7401C3
:10061000F090DF3C7480F090DF3D7494F022120182
:10062000201201A81201C11201341204F0D2AF75D8
:10063000440075370185370890004475F040120377
:100640000274F42521FA74013522FBE43523FCE41D
:100650003524FD7401B52A02800FC3EA9521EB957C
:1006600022EC9523ED952450EAE53E600E75440496
:10067000853E45753702753E008006754400753726
:1006800001E52B60B075080490004475F04012013C
:10069000F674F42521FA74013522FBE43523FCE4D9
:1006A0003524FD7406B5350280187405B535028011
:1006B000D4C3EA9521EB9522EC9523ED952450E3E4
:1006C00080C3752B00753F37754000754140900021
:0A06D0004475F0401203EE020635F7
:0600B200E478FFF6D8FD22
:100090007900E94400601B7A00900713780075939B
:1000A000F0E493F2A308B800020593D9F4DAF275EC
:0200B00093FFBC
:1006DA0020F71030F6118883A88220F507F6A88340
:0906EA0075830022F280F7F02272
:1000B8007800E84400600A79007593F0E4F309D801
:1000C800FC7800E84400600C790090F000E4F0A3AC
:0400D800D8FCD9FA7D
:0D00830075814712070FE582600302007EC1
:1006F30020F71430F6148883A88220F507E6A88330
:1007030075830022E280F7E49322E02275820022BF
:00000001FF
